:020000040000FA
:020000000428D2
:08000800831285010730990005
:100010008B138316FF239000F83085008312013084
:10002000AC00B1209420FD207430E1204030E1206C
:100030003C302C02031D2328B630E120B030E120F3
:10004000F330E1202A28B0302C07E120F330E12002
:10005000A030E120F4207920FD207430E1204030F0
:10006000E120D230E120D030E120CD30E120BA30A3
:10007000E120F4206C21A6202C087E2110100E080F
:10008000A6000F08A7002B102730A8001030A900E9
:100090005E200330A800E830A9005E20A80164308B
:1000A000A9005E20A8010A30A9005E20A801013045
:1000B000A9002B145E20851D0A211228AA012808F8
:1000C0002702031C7228031D692829082602031C25
:1000D00072282808A7022908A602031CA703AA0A57
:1000E0002B145F28B0302A072B1CA030A5009D20C0
:1000F0000800FD207430E1208030E1200230E12052
:10010000F4200800FD207430E1208030E12001302F
:10011000E120F4200800FD207430E1208030E1204F
:100120008530E120F4200800FD207430E12080308B
:10013000E1208C30E120F4200800FD207430E12023
:100140004030E1202508E120F420080090018E01D4
:100150008F018B0183168C0183128C010330900078
:100160000800FD207430E1200030E1200130E12062
:100170002130E120A030E1200730E1202430E120CF
:100180000F30E1200630E120FD207430E120803086
:10019000E1204030E1204030E1201830A300003061
:1001A000E120A30BCF28F420FD207430E1200030A3
:1001B000E1203030E1200130E1200C30E120F4205A
:1001C0000800A4000830A20085106C21A41B0514AF
:1001D000A41F05106C2185146C2185106C21A40DC1
:1001E000A20BE4280521080005106C2185146C2160
:1001F00005146C2185106C210800051485146C21F0
:1002000005106C2185106C21080085146C21851067
:100210006C2108008220FD207430E1204030E12074
:10022000C230E120E130E120FA30E120E130E1208C
:10023000BA30E120B0302C07E120F330E120A030CB
:10024000E120F42071218519612901302C02031D60
:100250003B290630AC008B206C21FD207430E1205E
:100260004030E120B0302C07E120F330E120A03015
:10027000E120F420612906302C02031D50293C3076
:10028000AC008B206C21FD207430E1204030E12057
:10029000B630E120B030E120F330E120F4206129D4
:1002A0000130AC008B206C21FD207430E120403007
:1002B000E120B0302C07E120F330E120A030E12034
:1002C000F4207121851D25297121851D2529712184
:1002D000851D2529822008001030A100A10B6E2960
:1002E0000800FF30A000FF30A10000000000000067
:1002F0000000A10B7529A00B73290800A300851D20
:1003000090290430A200FA30A000FA30A1000000C9
:10031000A10B8729A00B8529A20B8329A30B7F2979
:020320000800D3
:0207FE005C3469
:02400E00843FED
:00000001FF
